:100000000C9432080C9452080C9452080C94520828
:100010000C9452080C9452080C9452080C945208F8
:100020000C9452080C9452080C9452080C945208E8
:100030000C9452080C9452080C9452080C945208D8
:100040000C9452080C94FB120C9452080C94520815
:100050000C9452080C9452080C9452080C945208B8
:100060000C9452080C947B290C9447290C94520848
:100070000C9452080C9463080C9452080C94520887
:100080000C9452080C9452080C9452080C94520888
:100090000C9452080C9452080C9452080C94520878
:1000A0000C9452080C9452080C9452080C94520868
:1000B0000C9452080C9452080C9452080C94520858
:1000C0000C9452080C9452080C9452080A7377202E
:1000D000310A000A737720300A00414D433A206EFE
:1000E0006F77204D300A00414D433A206E6F7720E4
:1000F0004D310A00414D433A2068616E646C6520C1
:10010000636C6F7365640A00414D433A204D3120A2
:1001100068616E646C652073746174757320636FBD
:100120007272656374696F6E0A00414D433A206EC6
:100130006F77204D320A00414D433A2068616E646A
:100140006C65206F70656E65640A00414D433A200E
:100150006E6F77204D330A00414D433A2068616E3F
:10016000646C65206F70656E65640A00414D433AAA
:10017000206E6F77204D340A00414D433A2068616C
:100180006E646C65206F70656E65640A00414D4356
:100190003A204D342068616E646C6520737461741C
:1001A000757320636F7272656374696F6E0A0041C4
:1001B0004D433A206E6F77204D350A00414D433A4A
:1001C0002068616E646C6520636C6F7365640A00FF
:1001D000414D433A206E6F77204D360A000A414D5B
:1001E00043206873776170206F75743A20000A535A
:1001F0004953383330300A004275696C742077698E
:100200007468204156522D4743433A2000342E361D
:100210002E320020616E64204156522D4C494243DB
:100220003A2000312E382E30002072656C656173E3
:10023000653A20003230313131323238000A6F6E87
:100240002000536570202039203230313300202FB8
:10025000200031353A33303A3539000A0A00414D31
:1002600043207374617475733A204D000A00525430
:100270004D207374617475733A204D000A0A002092
:10028000436F6D6D616E646C6973743A0A205354E8
:100290004154202D204669726D7761726520526548
:1002A000766973696F6E2C205374617475732C209A
:1002B0006574632E2E2E0A2048454C50202D207444
:1002C00068697320706167650A002072746D207A16
:1002D0006F6E65333A200020616D63207A6F6E6522
:1002E000333A20002072746D206D617463683A2087
:1002F000002072746D20636C6F7365640A00207255
:10030000746D206F70656E65640A002072746D20D4
:100310006F70656E65640A002072746D206F706581
:100320006E65640A002072746D206F70656E65647E
:100330003A2000505752202B3132563A2000206D7F
:10034000560A4420202B332E33563A202000206DAD
:10035000560A4420202B312E30563A202000206DA2
:10036000560A4420202B312E38563A2020002045B2
:1003700072617375726520454550524F4D202E2E87
:100380002E2000205772697465204144353333387C
:100390003A200020526561642041443533333800EF
:1003A0000A454550524F4D205345524E554D3A2027
:1003B000000A0069326320627573206572726F7281
:1003C0000A00756E6B6E6F776E20693263207374EE
:1003D0006174652000657272207374613A20006553
:1003E000727220736C613A200065727220647461CD
:1003F0003A20000A0A53495338333030206465628A
:1004000075672070726F6D70740A000A0A626F6FF0
:100410007476616C7565203D20000A000A0A534914
:1004200053383330302064656275672070726F6DA9
:1004300070740A005744544353523A20000A004D46
:100440004D432046573A20000A4275696C74207764
:10045000697468204156522D4743433A2000342E98
:10046000362E320020616E64204156522D4C494296
:10047000433A2000312E382E30002072656C6561C1
:1004800073653A20003230313131323238000A6F30
:100490006E20005365702020392032303133002027
:1004A0002F200031353A33313A3032000A004D43C3
:1004B0005553523A20000A007265737461727420B9
:1004C000616674657220636F6C6420726573657415
:1004D0000A004D4F4453544154455F504F574552C5
:1004E0004544202D3E204D4F4453544154455F57C1
:1004F0004149545F524553455420000D0A004D4F69
:100500004453544154455F574149545F5245534504
:1005100054202D3E204D4F4453544154455F574184
:1005200049545F465047415F444F4E4520000D0AF5
:10053000004D4F4453544154455F574149545F4621
:100540005047415F444F4E45202D3E204D4F445370
:10055000544154455F465047415F52445920000D75
:100560000A004D4F4453544154455F465047415F44
:1005700052445920000D0A00708A728E9290748C39
:1005800076989C9AA0A4889E868478947A96828095
:100590007C7EA20700510131000006C10003540215
:1005A00001FF7F00703F0000040000620200040CA5
:1005B000C0077FEFABFF00F7F2E9A2A7AB02020092
:1005C0000000C6442B312E38560000000000000009
:1005D0000000000600510131000005C10003540273
:1005E00001FF7F00703F0000040000620200040C65
:1005F000C0077FEFABFF00F7F2E9A2A7AB02020052
:100600000000C6442B312E305600000000000000D0
:100610000000000200510130000001C1000355013B
:1006200001FF7F00703F0080010000010600040C04
:1006300000001946007DC9555046D8DDE705050084
:100640000000C57446504741000000000000000053
:1006500000000000005112150000002B000000C037
:100660000000CA5349533833303052544D000051C2
:1006700012120000002B000000C10000C7534953B4
:1006800038333030020051012F000008C0000354FD
:100690000101FF7F00703F0080010000010600049F
:1006A0000C00001946007DC9555046D8DDE7050508
:1006B000000000C47452544D00000000000000000F
:1006C000000000000100510135000007C000034098
:1006D000F26F0700000007000000000000000000AB
:1006E000000000000000000000000000000000000A
:1006F000000000CA486F745377617052544D000077
:10070000000000000500510131000004C100035445
:100710000201FF7F00703F0000040000A1020004FE
:100720000CC0077FEFABFF00F7F2E9A2A7AB020214
:10073000000000C6442B332E33560000000000009A
:10074000000000000400510132000003C100035406
:100750000201FF7F00703F00000400003602000429
:100760000CD0077FEFABFF00F7F2E9A2A7AB0202C4
:10077000000000C75057522B3132560000000000D5
:10078000000000000300510131000002C1000354C9
:100790000101FF7F00703F0080010000010600049E
:1007A0000C00001946007DC9555046D8DDE7050507
:1007B000000000C674506F776572000000000000F2
:1007C000000000000100510132000000C1000340A0
:1007D000F26F0700000007000000000000000000AA
:1007E0000000000000000000000000000000000009
:1007F000000000C7486F745377617000000000006C
:100800000000000070726F633A204E4554464E5F00
:100810004150503A20434D445F4745545F4445564C
:100820004943455F49440A0070726F633A204E4560
:1008300054464E5F53454E535F4556454E543A20FD
:10084000434D445F5345545F4556454E545F5245B2
:100850004345495645520A0070726F633A204E452F
:1008600054464E5F53454E535F4556454E543A20CD
:10087000434D445F4745545F4556454E545F52458E
:100880004345495645520A0070726F633A204E45FF
:1008900054464E5F53454E535F4556454E543A209D
:1008A000434D445F504C4154464F524D5F45564571
:1008B0004E540A0070726F633A204E4554464E5FA4
:1008C00053454E535F4556454E543A20434D445F81
:1008D0004745545F4445564943455F5344525F4939
:1008E0004E464F0A0070726F633A204E4554464E92
:1008F0005F53454E535F4556454E543A20434D4451
:100900005F4745545F4445564943455F5344520A47
:100910000070726F633A204E4554464E5F53454E09
:10092000535F4556454E543A20434D445F5245531C
:100930005F4445564943455F5344525F5245500A10
:100940000070726F633A204E4554464E5F53454ED9
:10095000535F4556454E543A20434D445F474554F6
:100960005F53454E534F525F52454144494E470AEB
:100970000070726F633A204E4554464E5F53454EA9
:10098000535F4556454E543A20756E6B6E6F776EC9
:100990003A200070726F633A204E4554464E5F53C2
:1009A000544F524147453A20434D445F4745545FB9
:1009B0004652555F494E565F415245415F494E464A
:1009C0004F0A0070726F633A204E4554464E5F5393
:1009D000544F524147453A20434D445F52454144AC
:1009E0005F4652555F444154413A2000414D430A0D
:1009F0000052544D0A0070726F633A204E455446BF
:100A00004E5F53544F524147453A20434D445F5740
:100A1000524954455F4652555F444154413A200083
:100A2000414D430A0052544D200070726F633A20CA
:100A30004E4554464E5F5049434D473A20434D443E
:100A40005F4745545F5049434D475F50524F5053A5
:100A50000A0070726F633A204E4554464E5F50490B
:100A6000434D473A20434D445F4652555F434F4EF6
:100A700054524F4C3A2000414D430A0052544D0A03
:100A80000070726F633A204E4554464E5F504943A2
:100A90004D473A20434D445F4745545F4652555FAA
:100AA0004C45445F50524F50530A0070726F633A86
:100AB000204E4554464E5F5049434D473A20434DE2
:100AC000445F4745545F4C45445F434F4C4F525F32
:100AD00043415041420A0070726F633A204E4554C0
:100AE000464E5F5049434D473A20434D445F53457E
:100AF000545F4652555F4C45445F53544154450A38
:100B00000070726F633A204E4554464E5F50494321
:100B10004D473A20434D445F4745545F4652555F29
:100B20004C45445F53544154450A0070726F633A18
:100B3000204E4554464E5F5049434D473A20434D61
:100B4000445F4745545F4652555F4C45445F53549C
:100B5000415445206572723A000A0070726F633A20
:100B6000204E4554464E5F5049434D473A20434D31
:100B7000445F4745545F4445565F4C4F4341545F83
:100B80005245435F49440A0070726F633A204E45F4
:100B900054464E5F5049434D473A20434D445F46CB
:100BA00052555F434F4E54524F4C5F434150414268
:100BB0000A0070726F633A204E4554464E5F5049AA
:100BC000434D473A20434D445F5345545F414D43A5
:100BD0005F504F52545F53544154450A0070726F36
:100BE000633A204E4554464E5F5049434D473A20A4
:100BF000434D445F4745545F414D435F504F52540E
:100C00005F53544154450A0070726F633A204E4559
:100C100054464E5F5049434D473A20434D445F4749
:100C200045545F434C4F434B5F53544154450A0076
:100C300070726F633A204E4554464E5F5049434DA3
:100C4000473A20434D445F5345545F4652555F41F8
:100C5000435449564154494F4E0A0070726F633AEB
:100C6000204E4554464E5F5049434D473A20434D30
:100C7000445F5345545F504F5745525F4C4556456E
:100C80004C0A0070726F633A204E4554464E5F50D6
:100C900049434D473A20756E6B6E6F776E0A007050
:100CA000726F633A204E4554464E5F56454E444F50
:100CB000523A20434D445F524541445F52544D5F88
:100CC00045450A0070726F633A204E4554464E5FA8
:100CD00056454E444F523A20434D445F5752495473
:100CE000455F52544D5F45450A0070726F633A206C
:100CF0004E4554464E5F56454E444F523A20434D62
:100D0000445F4D4F444946595F52544D5F45455FDE
:100D100057500A0070726F633A204E4554464E5F3A
:100D200056454E444F523A20434D445F5345545F1D
:100D3000464C4153485F424F4F545F5245560A005C
:100D400070726F633A204E4554464E5F56454E448E
:100D50004F523A20434D445F52455345545F4650ED
:100D600047410A0070726F633A204E4554464E5F09
:100D700056454E444F523A20434D445F4745545FD9
:100D80004649524D575F56455253494F4E0A0070DF
:100D9000726F633A204E4554464E5F56454E444F5F
:100DA000523A20434D445F4745545F754457435F73
:100DB0004441435F56414C55450A0070726F633A97
:100DC000204E4554464E5F56454E444F523A2043BE
:100DD0004D445F5345545F754457435F4441435FFF
:100DE00056414C55450A0070726F633A204E455487
:100DF000464E5F56454E444F523A20464F4F200ACA
:100E00000052544D3A206E6F77204D300A005254F4
:100E10004D204D61736B3A200052544D3A2045529B
:100E2000524F523A20493243206275732053444155
:100E300020737475636B206C6F770A0052544D3ABF
:100E4000206E6F77204D310A000A636F6D706174F8
:100E50006962696C69747920636865636B3A200024
:100E60002D3E20737563636573730A002D3E206EFB
:100E70006F206D61746368657320666F756E640AB8
:100E80000052544D204D61736B3A20000A005254B9
:100E90004D3A2068616E646C6520636C6F736564A5
:100EA0002C20656467650A0052544D3A2068616ED3
:100EB000646C6520636C6F7365642C204D30206C0E
:100EC0006576656C0A0052544D3A206D6F64756CFE
:100ED000652072656D6F7665640A0052544D3A2044
:100EE0006E6F77204D320A0052544D204D61736B66
:100EF0003A200052544D3A2068616E646C65206F50
:100F000070656E65640A0052544D3A206D6F6475C9
:100F10006C652072656D6F7665640A0052544D3AB7
:100F2000206E6F77204D330A0052544D3A206E6F79
:100F300077204D340A0052544D204D61736B3A2096
:100F40000052544D3A205365747570204457435FE6
:100F500044414320746F203256350A0052544D3AB2
:100F60002068616E646C65206F70656E65640A0050
:100F700052544D3A206D6F64756C652072656D6FCB
:100F80007665640A0052544D3A20536574646F7755
:100F90006E204457435F4441430A0052544D3A2067
:100FA0006E6F77204D350A0052544D204D61736BA2
:100FB0003A200052544D3A20536574646F776E2086
:100FC0004457435F4441430A0052544D3A206D6FE9
:100FD00064756C652072656D6F7665640A005254A5
:100FE0004D3A206E6F77204D360A0052544D204DF9
:100FF00061736B3A200052544D3A206D6F64756CEA
:10100000652072656D6F7665640A000A616D632004
:10101000776974686F7574207A33207265636F72B4
:1010200064730A000A72746D20776974686F75744E
:10103000207A33207265636F7264730A000A666FE8
:101040007220616D633A2000666F722072746D3A8F
:1010500020000A52544D206873776170206F7574B8
:101060003A20000011241FBECFEFD1E2DEBFCDBF7A
:1010700013E0A0E0B2E0E2E1FBE500E00BBF02C05C
:1010800007900D92AA3BB107D9F71BBE17E0AAEB58
:10109000B3E001C01D92AC31B107E1F70E94632AB1
:1010A0000C94872D0C9400001092F30310927C0096
:1010B00087EC80937A0080917A0084FFFCCF8FECDC
:1010C00080937A0008951F920F920FB60F920BB67D
:1010D0000F9211242F934F935F936F937F938F936E
:1010E0009F93AF93BF93EF93FF938091780090917C
:1010F0007900A0E0B0E04091BA035091BB03609149
:10110000BC037091BD03840F951FA61FB71F80936A
:10111000BA039093BB03A093BC03B093BD0320918B
:10112000BE032F5F2093BE032223E9F42091F30333
:10113000E22FF0E0EE0FFF1FE551FC4F892F9A2FB1
:10114000AB2FBB27918380831092BA031092BB030D
:101150001092BC031092BD03822F8F5F8370809327
:10116000F30380937C008FEC80937A00FF91EF91E2
:10117000BF91AF919F918F917F916F915F914F91AF
:101180002F910F900BBE0F900FBE0F901F901895D0
:10119000E82FF0E0E370F070EE0FFF1FE551FC4F19
:1011A0008081918108951F93CF93DF93CDB7DEB7F0
:1011B000C354D0400FB6F894DEBF0FBECDBF182F7A
:1011C0008DED91E00E94B529812F0E942E2A80E0AA
:1011D00092E00E94A3298091F5058C8380E18D83A4
:1011E0008091AC058F838091F40588878C5F809314
:1011F000F40582E0898784E08A8782EF8B871C86EA
:101200008FE68D871E878BE08B83CE0101960E942F
:10121000A01381E08A83CE0101960E94751010937D
:101220000202CD5BDF4F0FB6F894DEBF0FBECDBF1D
:10123000DF91CF911F910895CF9380E80E94B42849
:10124000C82F80910402809303028091C50380938C
:1012500004028091C603C81749F0CC2319F08CEC26
:1012600090E002C083ED90E00E94B52980E80E94E2
:10127000B4289091C403882319F09D7F916002C027
:1012800092609E7F9093C40380910402833009F49E
:1012900082C0843040F490910302813071F1823039
:1012A00008F058C00AC0853009F4CDC0853008F474
:1012B00098C0863009F007C1EAC0992309F400C13B
:1012C0008AED90E00E94B52980E060E041E050E0C6
:1012D0000E94B31081E060E041E050E00E94B31052
:1012E00082E060E043E050E00E94B31082E060E002
:1012F00040E050E00E94B310E3C0913051F080E034
:1013000060E041E050E00E94B31087EE90E00E9460
:10131000B5298091C603C81771F0CC2361F0C09342
:10132000C60384EF90E00E94B52980E00E94D308B4
:1013300082E08093C5038091C603C81709F445C0B5
:10134000CC2309F042C01092C60388E091E00E94CD
:10135000B5293BC0923021F08AE291E00E94B52984
:101360008091C603C81771F0CC2361F41092C603B4
:1013700087E391E00E94B52981E00E94D30881E0D3
:101380008093C5038091C303882309F49CC0109205
:10139000C30383E096C080910302833021F08BE485
:1013A00091E00E94B5298091C603C81771F0CC2343
:1013B00061F41092C60388E591E00E94B52981E0AE
:1013C0000E94D30881E08093C5038091C2038823E3
:1013D00009F479C01092C20381E08093AB0584E0E8
:1013E00070C080910302843021F08CE691E00E946D
:1013F000B5298091C603C81771F0CC2361F410920F
:10140000C60389E791E00E94B52981E00E94D308D4
:1014100085E08093C5038091C603C81741F0CC23B3
:1014200031F0C093C6038DE891E00E94B529809108
:10143000C003882309F447C01092C00387E080935B
:10144000AB0586E03EC080910302853021F08FEA33
:1014500091E00E94B5298091C603C81771F0CC2392
:1014600061F0C093C6038CEB91E00E94B52980E047
:101470000E94D30884E08093C5038091C103882330
:1014800079F01092C10386E08093C50309C0809172
:101490000302863029F00D9A80ED91E00E94B52973
:1014A0008091C003882329F01092C00387E08093C5
:1014B000AB058091AB05882331F482E00E94D3080C
:1014C00081E08093C5038091BF03882331F0809130
:1014D00002020E94D3081092BF03CF910895809119
:1014E000040208958091C403089581E08093C303AA
:1014F000089581E08093C203089581E08093C10341
:10150000089581E08093C003089581E08093BF0334
:1015100008956F927F928F929F92AF92BF92CF92D7
:10152000DF92EF92FF920F931F93CF93DF93CDB78C
:10153000DEB7C850D1400FB6F894DEBF0FBECDBFA6
:101540004C01E62E3A01FC011082CE01019660E0CA
:1015500070E048E050E00E94572DFE01319697E080
:1015600080E02191820F9150E1F78195988589174C
:1015700009F059C00E8110E093E0000F111F9A95F9
:10158000E1F70115110509F450C089E0A82EB12C2E
:10159000AC0EBD1EB80160507040CE01019645E012
:1015A00050E00E94572D8A819981890FFB808F0D11
:1015B0009C81890F81959D818917C9F5CF2CDD24E8
:1015C0000B5F1F4FB80160507040C501A6010E941B
:1015D000572D20E030E006C08A0D9B1DFC01808164
:1015E000280F3F5F832F90E08C159D05A8F3219570
:1015F0008C812817F1F48C85803379F4F401808193
:101600008F5F80838E1549F46114710431F0C3013A
:10161000B5014F2D50E00E944E2D8A8187FD0BC0F1
:101620000C0D1D1DB7CF82E007C083E005C084E02C
:1016300003C085E001C080E0C85FDE4F0FB6F894BC
:10164000DEBF0FBECDBFDF91CF911F910F91FF90F5
:10165000EF90DF90CF90BF90AF909F908F907F9052
:101660006F900895EF92FF920F931F93CF93DF93A4
:10167000CDB7DEB728970FB6F894DEBF0FBECDBF4B
:101680007C01CE01019660E070E048E050E00E94ED
:10169000572DFE01319697E080E02191820F915005
:1016A000E1F781959885891749F50E8110E023E0CF
:1016B000000F111F2A95E1F70115110509F1B80175
:1016C00060507040CE01019645E050E00E94572DD9
:1016D0002A819981920F8B81980F3C81930F91956C
:1016E0003D81931779F490E00596080F191F27FFA5
:1016F000E6CFF7011183008380E005C082E003C0DC
:1017000083E001C084E028960FB6F894DEBF0FBED8
:10171000CDBFDF91CF911F910F91FF90EF90089572
:1017200088E193E00E94B52980E008958FE792E078
:101730000E94B52980E00895CF93DF9300D0CDB704
:10174000DEB783E993E00E94B5298CE061E0AE0149
:101750004F5F5F4F0E940E27882329F085E092E0BB
:101760000E94A3290AC08DE092E00E94A3298981EA
:101770000E942E2A8A810E942E2A82E192E00E94F3
:10178000A32980E00F900F90DF91CF910895CF9320
:10179000DF9300D000D0CDB7DEB719821A821B824A
:1017A0001C828CE289838CE18A83AAE2B4E0FE0188
:1017B000319680E090E03D91232F20532A3008F0AD
:1017C00027502193019684309105A9F7898182954C
:1017D000807F9A819F70892B89838B818295807FFE
:1017E0009C819F70892B8A8383E893E00E94B529AE
:1017F00089810E942E2A8A810E942E2A8CE061E033
:10180000AE014F5F5F4F0E946124882319F084E18D
:1018100092E002C080E292E00E94A32980E00F9053
:101820000F900F900F90DF91CF910895CF93DF939A
:101830008EE693E00E94B529C0E0D0E080E5BE01CD
:1018400040E00E946723219682E0C030D807B1F7BC
:101850008BE292E00E94A32980E0DF91CF9108956E
:10186000EF92FF920F931F93CF93DF9300D000D09E
:1018700000D0CDB7DEB782E392E00E94A32981E5D4
:101880006AEF70E046E050E09E012F5F3F4F0E94FC
:10189000C423882329F084E492E00E94A32910C085
:1018A0007E010894E11CF11C00E010E0F701819139
:1018B0007F010E942E2A0F5F1F4F06301105B1F7DE
:1018C00082E192E00E94A32980E026960FB6F89468
:1018D000DEBF0FBECDBFDF91CF911F910F91FF9063
:1018E000EF900895CF93DF9380E00E94C808EC0149
:1018F00083E393E00E94B529BE0180E090E020E000
:101900003AE84DE050E00E94E62C0E94E52981E093
:101910000E94C808EC018EE393E00E94B529BE0145
:1019200080E090E020E835E044E050E00E94E62CC2
:101930000E94E52982E00E94C808EC018EE493E051
:101940000E94B529BE0180E090E020E031E742E04E
:1019500050E00E94E62C0E94E52983E00E94C8081E
:10196000EC018EE593E00E94B529BE0180E090E095
:1019700020E031E742E050E00E94E62C0E94E52999
:101980008EE492E00E94A32980E0DF91CF91089538
:10199000EF92FF920F931F93CF93DF9300D0CDB7B9
:1019A000DEB785E293E00E94B529CE0101960E9440
:1019B000692190E00E94E52903E512E0C8010E9438
:1019C000A32989819A810E94E52922E1E22E22E061
:1019D000F22EC7010E94A329CE0101960E94320B6C
:1019E00090E00E94E529C8010E94A32989819A817B
:1019F0000E94E529C7010E94A32980E00F900F9063
:101A0000DF91CF911F910F91FF90EF9008958BE0A0
:101A100093E00E94B52986E00E94011F80E00895AE
:101A20008EEF92E00E94B52981E00E94011F80E0C4
:101A3000089581EF92E00E94B52980E00E94011F85
:101A400080E0089584EE92E00E94B5290E948222EF
:101A500090E00E94E52982E192E00E94A32988E0BB
:101A60000E94011F80E00895CF93DF930F92CDB7BE
:101A7000DEB787ED92E00E94B529CE01019660E0C5
:101A800040E050E00E94890A90E00E94E52983E549
:101A900092E00E94A329898190E00E94E52982E1D9
:101AA00092E00E94A32987E00E94011F80E00F902E
:101AB000DF91CF910895CF93DF930F92CDB7DEB72B
:101AC0008AEC92E00E94B529CE01019660E040E0E8
:101AD00050E00E94D72190E00E94E52983E592E042
:101AE0000E94A329898190E00E94E52982E192E089
:101AF0000E94A32985E00E94011F80E00F90DF91E2
:101B0000CF9108958EEE91E00E94B52988EF91E083
:101B10000E94B5298DE092E00E94B52983E192E010
:101B20000E94B52983E292E00E94B52989E292E001
:101B30000E94B52984E392E00E94B5298DE392E0EA
:101B40000E94B52982E492E00E94B5298EE492E0D9
:101B50000E94B52982E592E00E94B5298BE592E0CA
:101B60000E94B5298EE592E00E94B5290E946F0A75
:101B700090E00E94E5298CE692E00E94B5298EE66D
:101B800092E00E94B5290E94E91E90E00E94E5299A
:101B90008CE792E00E94B52980E0089585E592E007
:101BA0000E94A329109224040895CF93DF93AC01DF
:101BB000A0E08A2F90E0880F991F880F991FFC01E1
:101BC000E154FD4F60817181B0E02B2F30E0FB01CB
:101BD000E20FF31FE081EE2359F0240F351FE901D6
:101BE00028812E272F7511F4BF5FEFCFAF5FE1CFB4
:101BF000BB2349F081549D4FDC011296ED91FC917D
:101C00001397099501C081E0DF91CF910895CF939B
:101C1000DF930F92CDB7DEB7CE0101960E9429293E
:101C2000882309F04CC08981883019F08D3081F506
:101C300010C080912404882309F441C0815080930E
:101C4000240488E00E940A2980E20E940A2988E090
:101C500034C08AE00E940A298DE00E940A29E0919E
:101C60002404EE2371F0F0E0EB5DFB4F108285E27F
:101C700094E00E94D50D882321F08EE592E00E9429
:101C8000A329109224048FE692E00E94A32917C092
:101C90008B31A9F090912404903270F40E940A29AB
:101CA00080912404E82FF0E0EB5DFB4F9981908355
:101CB0008F5F8093240403C087E00E940A290F905D
:101CC000DF91CF910895CF92DF92EF92FF9286E35A
:101CD00090E00E94672D90E08F70907024E630E0D5
:101CE000829F6001839FD00C929FD00C1124EE2420
:101CF000D7FCE094FE2C87E390E00E94672D90E0F3
:101D00008F7090709C01220F331F63E0880F991F22
:101D10006A95E1F7280F391FC901AA2797FDA095F9
:101D2000BA2FC80ED91EEA1EFB1E88E390E00E945F
:101D3000672D8F70C80ED11CE11CF11C80EA93E066
:101D40000E94B52980E00E942E2A80E00E942E2A5F
:101D50008D2D0E942E2A8C2D0E942E2A81EB93E03D
:101D60000E94B5295A988FE99FE00197F1F700C0CA
:101D700000005A9A20E230E080E090E0A0E0B0E875
:101D80005B98AC01BD014C215D216E217F21411585
:101D900051056105710509F05B9AF8945A985A9AB1
:101DA0007894B695A795979587952150304041F73F
:101DB000FF90EF90DF90CF90089594E29093B80059
:101DC0008E7F8093BA001092BD0084E48093BC00A3
:101DD00010924F0410924E040895CF938091BC004E
:101DE00087FF67C0C091B900C87FC03661F0C136B7
:101DF00020F4CC2309F448C051C0C038D1F0C03A17
:101E000009F04CC02BC01092C903E091AF05F091CE
:101E1000B00580818068808380818E7F80838091FF
:101E2000BB00838381E08093C90394EC9093BC0052
:101E300012C0E091AF05F091B0058091C903909177
:101E4000BB00E80FF11D93838F5F8093C90384EC7F
:101E50008093BC0081E08093C8032BC0E091AF0564
:101E6000F091B0058091C903828380818160808375
:101E700080818F77808384EC8093BC001092C803AC
:101E80008AE080931A0315C083EB93E00E94B52982
:101E90008091BC0080698093BC000BC082EC93E011
:101EA0000E94B5298C2F0E942E2A8FEF92E00E946B
:101EB000A3298091C803CF910895CF92DF92FF921A
:101EC0000F931F93CF93DF930F92CDB7DEB780911F
:101ED000C703882341F490914F0480914E049817D2
:101EE00009F062C0F9C08F3F39F484E60E94D5281A
:101EF0008EEF8093C703F0C08E3F09F055C08091EC
:101F00005C05882311F140914E0450E023E430E059
:101F1000429FC001439F900D529F900D1124805B02
:101F20009B4F0E94B11E90914D04891771F48091CE
:101F30004E048F5F80934E04843011F410924E044F
:101F40001092C70310925C05C7C00E94E528882341
:101F500009F4C2C08091CA0381508093CA038823C8
:101F600021F084E60E94D5281FC080914E048F5F27
:101F700080934E04843011F410924E0481E093E07B
:101F80000E94A3291092C703A7C0489B02C0499989
:101F900003C090931A0303C0815080931A038AE10F
:101FA0008A95F1F700C001C09AE080911A03882356
:101FB00061F784EA8093BC008091BC0087FFFCCF6E
:101FC0001091B900187F183059F085ED93E00E9408
:101FD000B529812F0E942E2A8FEF92E00E94A3291B
:101FE00020914E0430E083E490E0289FF001299F87
:101FF000F00D389FF00D1124E05BFB4F838180933F
:10200000BB0084E88093BC008091BC0087FFFCCFBC
:102010001091B900187F183159F08FED93E00E94AC
:10202000B529812F0E942E2A8FEF92E00E94A329CA
:1020300011E083E4C82ED12C94E8F92E04E923C0E2
:10204000181719F40093BC001DC0E10FF11D838126
:102050008093BB00F092BC008091BC0087FFFCCF56
:102060002091B900287F283269F089EE93E0298316
:102070000E94B5292981822F0E942E2A8FEF92E09B
:102080000E94A3291F5F20914E04822F90E08C9D17
:10209000F0018D9DF00D9C9DF00D1124E05BFB4F38
:1020A0008281811768F68181813059F48091C7035C
:1020B0008E3F79F08FEF8093C70383E08093CA034C
:1020C00008C0822F8F5F80934E04843011F41092E9
:1020D0004E0484EC8093BC000F90DF91CF911F9150
:1020E0000F91FF90DF90CF90089560914F04462F9D
:1020F00050E023E430E0429FF001439FF00D529FF7
:10210000F00D1124E05BFB4FDC0183E40D900192A4
:102110008150E1F76F5F60934F04643011F41092C7
:102120004F0480E0089591E090935C0580934D0406
:102130000895DA01A90190E026E130E0829FF001E4
:10214000839FF00D929FF00D1124E35AFA4F61879F
:1021500010861286B183A083128213825583448332
:1021600016821782089590E026E130E0829FD00128
:10217000839FB00D929FB00D1124A35ABA4F6623CE
:10218000D1F412968C91129790E0880F991FED91DF
:10219000FC911197E80FF91F5183408312968C919F
:1021A00012978F5F12968C9312978430F1F41296E7
:1021B0001C921297089516968C91169790E0880FAE
:1021C000991F1496ED91FC911597E80FF91F518313
:1021D000408316968C9116978F5F16968C93169760
:1021E000843019F416961C9216970895CF93DF93B6
:1021F000EA0190E026E130E0829FD001839FB00D9C
:10220000929FB00D1124A35ABA4F662309F5139675
:102210008C91139712969C9112978917D9F190E09F
:10222000880F991FED91FC911197E80FF91F80819C
:1022300091819983888313968C9113978F5F13965E
:102240008C931397843041F513961C92139724C0F6
:1022500017968C91179716969C9116978917D1F01F
:1022600090E0880F991F1496ED91FC911597E80F57
:10227000F91F808191819983888317968C91179794
:102280008F5F17968C931797843031F417961C92B2
:10229000179702C081E001C080E0DF91CF910895DF
:1022A000EF92FF920F931F93CF93DF9300D0CDB7A0
:1022B000DEB7F82E282F30E086E190E0289F8001DD
:1022C000299F100D389F100D1124035A1A4FF80141
:1022D0008085882309F0BCC08285813041F081303F
:1022E00068F0823089F0833009F04BC028C025B1F6
:1022F000F80191859095922395B942C085B1F80176
:102300009185892B85B93BC0F8018585882349F0E3
:1023100095B181858095892385B98585815085878B
:102320000BC0F8018685882339F085B19185892B0A
:1023300085B9868581508687F80186851AC0F8019F
:102340008685882341F085B19185892B85B986855D
:10235000815086870CC0F8018585882341F095B1AE
:1023600081858095892385B9858581508587F80188
:102370008585882331F4838585878485868781E0F8
:102380008787F801E784F1E0EF1609F0CEC08F2DC2
:1023900061E0AE014F5F5F4F0E94F610882321F588
:1023A000F801E08649815A81CA019070009711F4C2
:1023B000108A4BC09C01215030402A3F310540F427
:1023C00082E0F801808B518B428B538B448B3DC054
:1023D0008C3F910519F4F801108637C08F3F9105A5
:1023E000A1F5F801E08A31C08F2D60E0AE014F5FAA
:1023F0005F4F0E94F610882341F589819A81907081
:102400008130910551F08130910550F08230910575
:1024100051F083309105C9F40FC0F801E28615C070
:10242000F801128612C09AE0F80193878AE5848742
:102430009587868782E008C09AE5F80193878AE04D
:1024400084879587868783E08287F80117866DC029
:10245000F8018089813039F0813060F0823081F07C
:10246000833081F519C025B1F801918590959223AB
:1024700095B927C085B1F8019185892B85B920C010
:10248000F8018489882341F085B19185892B85B92C
:1024900084898150848B0CC0F8018389882341F0A2
:1024A00095B181858095892385B983898150838BF6
:1024B000F8018389882331F48189838B8289848B15
:1024C00081E0858BF8018589882379F18F2D61E082
:1024D000AE014F5F5F4F0E94F610882321F561E047
:1024E000F801608749815A81CA019070009711F400
:1024F000108A19C09C01215030402A3F310540F418
:1025000082E0F801808B518B428B538B448B0BC044
:102510008C3F910519F4F801108605C08F3F910595
:1025200011F4F801608BF801158A0F900F90DF917C
:10253000CF911F910F91FF90EF900895DB0190E0F4
:1025400026E130E0829FF001839FF00D929FF00D15
:102550001124E35AFA4F80858C93828511968C93CF
:102560001197848512968C931297838513968C937A
:102570001397808914968C931497828915968C935F
:102580001597818916968C9316970895CF92DF92AE
:10259000EF92FF920F931F93CF93DF930F92CDB7DC
:1025A000DEB77B0189830E94EC27898181600E94CC
:1025B0000F28882321F40E94042881E012C081E0C2
:1025C0000E944428182F00E080E00E944428C82E72
:1025D000DD24C02AD12A0E940428F701D182C082BA
:1025E00080E00F90DF91CF911F910F91FF90EF90BE
:1025F000DF90CF9008951F920F920FB60F920BB6F7
:102600000F9211242F933F934F935F936F937F9378
:102610008F939F93AF93BF93EF93FF930E94742880
:102620008091CB039091CC0301969093CC0380933F
:10263000CB0323E0883E920739F481E08093A20522
:102640001092CC031092CB038091CD038F5F8093C7
:10265000CD03843629F481E08093A3051092CD0345
:102660008091CE038F5F8093CE038A3071F40E94F5
:10267000EB2881E08093AE051092CE038091E803B1
:10268000882319F081508093E803FF91EF91BF9167
:10269000AF919F918F917F916F915F914F913F91FA
:1026A0002F910F900BBE0F900FBE0F901F9018959B
:1026B00085B1817F85B9209A28988FEC97E00197A2
:1026C000F1F700C0000021E0199B20E081E01A9B97
:1026D00080E091E01B9B90E0289AEFECF7E03197C7
:1026E000F1F700C0000063B141E01A9B40E031E027
:1026F0001B9B30E051E061FF50E0251322E0841382
:1027000082E0931392E0E82FEE0FE80FE20F89E0EA
:10271000989F902D1124E90FF0E0E858FA4F84912A
:10272000089590E08057904062E070E00E94112D83
:10273000862F0895FC018481869586958170089581
:10274000FC0183819481890F819585838281DF01DA
:1027500023E090E005C015963C911597930F2F5FED
:1027600011962817C0F3DF01A80FB11D919513969C
:102770009C9313978F5F82830895CF93DF93EC012F
:1027800088818E7F806888830E945D0F88818F7723
:10279000888380E0DF91CF910895FC01838194814B
:1027A000890F819595819817D9F4828190E00197DE
:1027B00053E040E008C02E0F3F1FD90113962C9123
:1027C0001397420F5F5F252F30E0281739079CF3DE
:1027D000E80FF91F41958381841721F082E0089565
:1027E00081E0089580E008959F92AF92BF92CF92CA
:1027F000DF92EF92FF920F931F93CF93DF93CDB7AA
:10280000DEB760970FB6F894DEBF0FBECDBF8C0168
:102810007B01FE013296A5E4B3E086E00D900192C3
:102820008150E1F7D80114969C911497292F269591
:1028300026952A3009F4B1C22B3040F4243009F433
:102840004DC0263011F00C946D1E08C02C3209F4D6
:10285000F9C3203311F00C946D1EECC7F801D0843D
:10286000F1E0DF1611F00C946D1E84E098E00E94F8
:10287000B529D80116968C911697F7018383179680
:102880009C91179714968C9114978C5F8C7F292FAD
:102890002370822B84838091AC05868314968C915F
:1028A000149783709C7F892B878318968C91189737
:1028B00080871186128681E88387D486158681E514
:1028C00086878BE287878DEB808B82E9818B128AEA
:1028D000138A83E8848B82E10C94AC1ED80118968D
:1028E0008C911897803209F49FC0813248F481306E
:1028F00009F446C0813088F0823009F045C26EC0CC
:10290000823209F45EC1823208F4BDC0873209F414
:1029100019C28D3209F038C284C188E298E00E9461
:10292000B529F80181858093F50582858093F605A8
:102930008681D70113968C931397978184818C5F3E
:102940008C7F292F2370822B14968C93149780915F
:10295000AC0516968C931697848183709C7F892B87
:1029600017968C931797808518968C9318971996BD
:102970001C920E94850A0E94FD1E87E00C94E01DB7
:1029800088E598E00E94B529D80116968C91169793
:10299000F701838317969C91179714968C9114973F
:1029A0008C5F8C7F292F2370822B84838091AC05D0
:1029B000868314968C91149783709C7F892B8783D0
:1029C00018968C911897808711868091F5058287DB
:1029D0008091F605838789E00C94AC1E88E898E026
:1029E0000E94B529D80116968C911697F70183831A
:1029F00017969C91179714968C9114978C5F8C7FE7
:102A0000292F2370822B84838091AC0586831496B2
:102A10008C91149783709C7F892B878318968C9157
:102A200018978087118667C284EB98E00E94B529C9
:102A3000D80116968C911697F701838317969C916F
:102A4000179714968C9114978C5F8C7F292F237085
:102A5000822B84838091AC05868314968C91149785
:102A600083709C7F892B878318968C918087118631
:102A70000E94D427D7011A968C931A9781E01B964F
:102A80008C931B97CCC085EE98E00E94B529F80185
:102A90008681D70113968C931397978184818C5FDD
:102AA0008C7F292F2370822B14968C9314978091FE
:102AB000AC0516968C931697848183709C7F892B26
:102AC00017968C931797808518968C93189719965C
:102AD0001C92A384BB24948580E0A82AB92AC584CB
:102AE00096840E94D4270197A816B90629F48FEF7F
:102AF000F7018287838708C0C5010196D7011A961E
:102B00008C931A971B969C93F501EE0FFF1FE55BC4
:102B1000FC4F0C2D10E060817181600F711FC701A7
:102B20000C96492D50E00E94382DB5E0BC1560F0A0
:102B3000C801890D911D8530910534F0F701E01B26
:102B4000F10B8091AC05818BE2E0AE16B104C8F4C4
:102B5000FDE0FC1570F1DD24C601890D911D8D305D
:102B600091053CF1F701EC19FD098091AC0590E06D
:102B70008057904062E070E00E94112D605A618F92
:102B800018C049E04C15A8F0DD24C601890D911D3F
:102B90008930910574F0F701EC19FD098091AC05BD
:102BA00090E08057904062E070E00E94112D605AE2
:102BB000658B892D875FD70112968C9312970C94A1
:102BC000901E81E199E00E94B529F8018681D70124
:102BD00013968C931397978184818C5F8C7F292F18
:102BE0002370822B14968C9314978091AC051696C3
:102BF0008C931697848183709C7F892B17968C9376
:102C00001797808518968C93189719961C92199788
:102C100081E01A968C931A971B961C921B9789E059
:102C2000CBCF81E499E00E94B529F8018681D701D4
:102C300013968C931397978184818C5F8C7F292FB7
:102C40002370822B14968C9314978091AC05169662
:102C50008C931697848183709C7F892B17968C9315
:102C60001797808518968C93189719961C92199728
:102C700081859AE012969C9312978430C9F1853031
:102C800058F4813009F1813098F0823001F18330BD
:102C900011F00C94901E1EC0863009F43FC086309F
:102CA000D8F18730E9F1883011F00C94901E48C0BB
:102CB000F701128680EC83870E94720AD7011C9666
:102CC0008C931C970C94901E8091A0050AC0809153
:102CD000A50515C080E00E94C80896958795969531
:102CE0008795F701828780E4838714860C94901E71
:102CF00081E00E94C8089695879596958795D7019B
:102D00001A968C931A9780E41B968C931B971C96AB
:102D10001C921C970C94901E82E0DDCF83E0E9CFDB
:102D2000F701128680EC83870E94EC1ED7011C9667
:102D30008C930E94EC1EF70195878BE00C94AC1EDF
:102D400080E2DDCFF8012681D70113962C931397EB
:102D500027819C5F9C7F322F3370932B14969C931A
:102D600014979091AC0516969C9316979481937046
:102D70002C7F922B17969C93179718968C931897E5
:102D800019961C9219971EC481E799E00E94B529F3
:102D9000F80180850E942E2A48C5D80118968C918A
:102DA0001897813109F452C0823109F4B2C08031E0
:102DB00009F093C783E999E0288B0E94B529F801AF
:102DC00081852889882351F08130D1F4288B0E9495
:102DD000E91E2889882311F483ED13C0D7011A96C0
:102DE0001C921A9782E01B968C931B971C961C9240
:102DF0001C9719961C92199712962C93129705C03E
:102E000089ECF701818787E08283D80116968C913F
:102E10001697F701838317969C91179714968C91B8
:102E200014978C5F8C7F292F2370822B8483809151
:102E3000AC05868314968C91149783709C7F892BA4
:102E4000878318968C91189780876AC783EC99E0DE
:102E50000E94B529D80116968C911697F7018383A5
:102E600017969C91179714968C9114978C5F8C7F72
:102E7000292F2370822B84838091AC05868314963E
:102E80008C91149783709C7F892B878318968C91E3
:102E90001897808711861A96AC901A97BB241B96B8
:102EA0009C911B9780E0A82AB92A1C96CC901C976D
:102EB000C28619968C911997882321F0813009F0E8
:102EC0002FC70EC08CEE99E00E94B529B501605065
:102ED0007040C7010B964C2D50E00E94572D16C034
:102EE00081EF99E00E94B5290E94E91E882329F408
:102EF00083EDF701818787E02FC79701255F3F4F5B
:102F000080E5B5014C2D50E00E940C218C2D885F8E
:102F100052CE86EF99E00E94B529F801C280F6EF03
:102F2000CF0ED8011A96AC901A97BB241B969C9191
:102F30001B9780E0A82AB92A19968C9119978823A3
:102F400021F0813009F05DC014C080E29AE00E9457
:102F5000B529F701C286B50160507040C8010C96D2
:102F60004C2D50E00E946F2DD70119961C92199795
:102F700048C085E29AE00E94B52987E393E00E9469
:102F8000A329C5010E94E5298DE393E00E94A329AE
:102F90008C2D90E00E94E52985E393E00E94A3290F
:102FA0000E94E91EF701882349F1C28611868CE749
:102FB000BE016F5F7F4F0E94721F8823B1F4698149
:102FC00061616F7769838CE70E94971F882311F0F6
:102FD000F70114C09801245F3F4F80E5B5014C2DE7
:102FE00050E00E949C23882361F0D7011A961C921E
:102FF0001A9783ED19968C93199703C0128683ED67
:103000008187D80116968C911697F70183831796BE
:103010009C91179714968C9114978C5F8C7F292F15
:103020002370822B84838091AC05868314968C91C7
:10303000149783709C7F892B878318968C9118979F
:10304000808789C6D80118968C9118978C3009F41E
:1030500068C38D30A8F4853009F4B7C0863030F4E9
:10306000882321F1843009F0C8C357C0873009F4A0
:10307000E2C0873008F4DCC0883009F0BEC361C10B
:10308000893109F415C38A3138F48D3009F4C3C28B
:10309000813109F0B2C375C38E3109F406C38D3294
:1030A00009F43CC38A3109F0A8C335C38AE29AE027
:1030B0000E94B529F8018681D70113968C93139746
:1030C000978184818C5F8C7F292F2370822B1496AB
:1030D0008C9314978091AC0516968C9316978481E7
:1030E00083709C7F892B17968C93179780851896F1
:1030F0008C93189719961C9219971A961C921A97E6
:1031000082E31B968C931B9781E01C968C931C97F3
:103110001D961C921D978BE04FCD82E59AE00E9490
:10312000B529F8018681D70113968C93139797815F
:1031300084818C5F8C7F292F2370822B14968C9333
:1031400014978091AC0516968C93169784818370A2
:103150009C7F892B17968C931797808518968C9354
:10316000189719961C9219971A961C921A9788E02C
:1031700012968C9312978285882321F0813009F072
:10318000E6C515C087E79AE00E94B529F801838556
:10319000882321F0843009F0DAC506C01092AB050F
:1031A00082E30E94BA28BCC50E94810AB9C58CE797
:1031B0009AE00E94B529D8011B968C911B97843008
:1031C00009F0C5C50E94F91EABC581E89AE00E94CE
:1031D000B529F8018681D70113968C9313979781AF
:1031E00084818C5F8C7F292F2370822B14968C9383
:1031F00014978091AC0516968C93169784818370F2
:103200009C7F892B17968C931797808518968C93A3
:10321000189719961C9219971A961C921A9787E07C
:103220001B968C931B971C961C921C978AE0C4CC0F
:103230008BEA9AE050C587ED9AE00E94B529F80123
:10324000248545858285882321F0813009F041C29B
:1032500027C0C22EDD24942F80E0C82AD92A838576
:103260008130B1F0813020F0823009F087C112C086
:1032700080E061E0A6010E94B3100E946F0A8230D4
:1032800009F027C2CC2009F024C20E94750A21C28D
:1032900081E001C082E061E0A6010E94B31019C282
:1032A000F8018385813081F0813018F0823049F552
:1032B00016C0222319F02F3F29F402C080E015C068
:1032C00080E01AC080E01BC0222319F02F3F29F4B0
:1032D00002C081E00AC081E00FC081E010C022235B
:1032E00019F02F3F59F407C082E060E040E020E091
:1032F0000E94B61EEEC182E061E0F8CF82E062E09B
:10330000F7CFD8018681F701838317969C91179791
:1033100014968C9114978C5F8C7F292F2370822BAD
:1033200084838091AC05868314968C911497837066
:103330009C7F892B878318968C91189780878CECBB
:1033400008C581E09BE00E94B52919820DC0F801F3
:10335000E80FF11D83810E942E2A83E493E00E94EE
:10336000A32989818F5F89838981D80112969C91D5
:103370001297891760F385E393E00E94A329F8016F
:103380008285882309F023C18385813009F44FC0E9
:10339000813020F0823009F0E4C08FC080E0BE01AF
:1033A000685F7F4F0E949E128985882319F08130C3
:1033B00071F404C0F701148615860EC08FEFD70193
:1033C0001C968C931C971D961C921D9705C08A8590
:1033D000F70184878B85858781E0D7011E968C93C2
:1033E0001E979CE012969C9312979885913009F055
:1033F000B5C082E01B968C931B978C85882319F0AF
:10340000813071F404C0F7011786108A0EC08FEF67
:10341000D7011F968C931F9750961C92509705C00A
:103420008D85F70187878E85808B81E08DC081E057
:10343000BE01685F7F4F0E949E128985882319F024
:10344000813071F408C0D7011C961C921C971D9600
:103450001C921D970EC08FEFF7018487158609C057
:103460008A85D7011C968C931C978B851D968C930F
:103470001D9782E0F70186879CE0928398859130C2
:10348000C9F483878C85882319F0813049F403C0FF
:103490001786108A09C08FEFF7018787108A04C04A
:1034A0008D8587878E85808B82E0F701818B8FE009
:1034B00082838DC081E083878AC082E0BE01685F1D
:1034C0007F4F0E949E128985882319F0813071F404
:1034D00004C0F701148615860EC08FEFD7011C9625
:1034E0008C931C971D961C921D9705C08A85F70129
:1034F00084878B85858783E0D7011E968C931E97E2
:103500008CE012968C9312978885813031F582E099
:103510001B968C931B978C85882319F0813071F44E
:1035200004C0F7011786108A0EC08FEFD7011F96CF
:103530008C931F9750961C92509705C08D85F7016C
:1035400087878E85808B83E0D70151968C93519726
:103550008FE012968C9312973AC081E0F70183872F
:1035600036C08BE29BE00E94B529D8011A968C9157
:103570000E942E2A89E59BE00E94B529F8018681E8
:10358000D70113968C931397978184818C5F8C7FDE
:10359000292F2370822B14968C9314978091AC055D
:1035A00016968C931697848183709C7F892B17962F
:1035B0008C931797808518968C9318978CEC199696
:1035C0008C9319971A961C921A9788E0F5CAF801FD
:1035D0008681D70113968C931397978184818C5F92
:1035E0008C7F292F2370822B14968C9314978091B3
:1035F000AC0516968C931697848183709C7F892BDB
:1036000017968C931797808518968C931897199610
:103610001C92199746C08BE59BE00E94B529F801E2
:103620008285882319F08130A1F40CC0D7011B9644
:103630001C921B971C961C921C9719961C9219970A
:103640008AE00DC0F7018387148611868AE08283A1
:1036500008C08CECD70119968C93199787E01296C5
:103660008C93F8018681D70113968C9313979781D9
:1036700084818C5F8C7F292F2370822B14968C93EE
:1036800014978091AC0516968C931697848183705D
:103690009C7F892B17968C931797808518968C930F
:1036A00018971A961C921A973BC388E89BE013C39D
:1036B00082EB9BE00E94B529F8018685882319F0EA
:1036C0000E94790A06C00E946F0A853011F40E9498
:1036D0007D0AD80116968C911697F7018383179669
:1036E0009C91179714968C9114978C5F8C7F292F3F
:1036F0002370822B84838091AC05868314968C91F1
:10370000149783709C7F892B878318968C911897C8
:10371000808711861FC38DED9BE0DDC288E09CE0B1
:10372000DAC280E39CE00E94B529D80116968C91FC
:103730001697F701838317969C91179714968C918F
:1037400014978C5F8C7F292F2370822B8483809128
:10375000AC05868314968C91149783709C7F892B7B
:10376000878318968C9118978087128688E08283C9
:103770001A968C911A978823A1F1813009F0D0C252
:10378000ABC18BE59CE00E94B529D80116968C91BF
:103790001697F701838317969C91179714968C912F
:1037A00014978C5F8C7F292F2370822B84838091C8
:1037B000AC05868314968C91149783709C7F892B1B
:1037C000878318968C9118978087128688E0828369
:1037D0001A968C911A97882321F0813009F0A0C2A3
:1037E00002C08FEF0CC1F8018385882319F00E9475
:1037F000F11E67C20E94F51E64C283E89CE00E942D
:10380000B52919820DC0F801E80FF11D83810E94CE
:103810002E2A83E493E00E94A32989818F5F898304
:103820008981F8019281891770F385E393E00E9402
:10383000A32953C2D80118962C911897233009F464
:10384000B4C0243030F4213089F0223008F05FC059
:1038500078C1253009F443C1253008F4F4C026307E
:1038600009F4B0C1273009F034C2ECC18FE99CE003
:103870000E94B529F801C1849284D384A4848681EE
:10388000D70113968C931397978184818C5F8C7FDB
:10389000292F2370822B14968C9314978091AC055A
:1038A00016968C931697848183709C7F892B17962C
:1038B0008C931797808518968C93189787E01296AB
:1038C0008C93B0E1BA1510F482E801C20E94E91E9F
:1038D000882309F493C0CC2011F490E5C92E692DFA
:1038E00070E09D2D80E0682B792B9701265F3F4F7C
:1038F0008C2D4A2D50E00E940C21882309F0A1C094
:10390000D70119961C9219978A2D895F55C984ECA5
:103910009CE00E94B529F801C184A284D384448527
:103920008681D70113968C931397978184818C5F3E
:103930008C7F292F2370822B14968C93149780915F
:10394000AC0516968C931697848183709C7F892B87
:1039500017968C931797808518968C93189787E005
:1039600012968C931297413110F082E849C0488B2F
:103970000E94E91E4889882311F480E8A8C1CC2060
:1039800011F480E5C82E6A2D70E09D2D80E0682B33
:10399000792B9801235F3F4F8C2D50E00E949C2390
:1039A000882309F499C081E82AC08AEE9CE00E942D
:1039B000B529D80116968C911697F701838317962F
:1039C0009C91179714968C9114978C5F8C7F292F5C
:1039D0002370822B84838091AC05868314968C910E
:1039E000149783709C7F892B878318968C9180878E
:1039F00087E082830E94E91E882331F480E8D701A2
:103A000019968C9319978CC18CE7BE016F5F7F4F1D
:103A10000E94721F8823A9F48981982F9161D8018F
:103A200019962C911997222311F0816902C0892FD0
:103A30008F7789838CE769810E94971F882309F417
:103A400040C181E844C184E19DE00E94B529F801AC
:103A50008681D70113968C931397978184818C5F0D
:103A60008C7F292F2370822B14968C93149780912E
:103A7000AC0516968C931697848183709C7F892B56
:103A800017968C931797808518968C93189787E0D4
:103A900012968C93129782B18C7F82B9818580FDBA
:103AA000119AF801818581FD109A8FEF9FE00E94A5
:103AB000672D8983D80119966C91199790E0262F6C
:103AC00030E08227932783709070009729F063700D
:103AD0008FEF9FE00E94792DF701118621C180E4CC
:103AE0009DE00E94B529D80116968C911697F70192
:103AF000838317969C91179714968C9114978C5FDB
:103B00008C7F292F2370822B84838091AC05868340
:103B100014968C91149783709C7F892B87831896B9
:103B20008C911897808787E08283389A8FEF99E687
:103B3000A8E181509040A040E1F700C00000389813
:103B4000C0C084E69DE00E94B529F8018681D701B6
:103B500013968C931397978184818C5F8C7F292F88
:103B60002370822B14968C9314978091AC05169633
:103B70008C931697848183709C7F892B17968C93E6
:103B80001797808518968C93189787E012968C93D8
:103B9000129719961C92199720E00FC0822F90E07F
:103BA000F701E80FF91F42E050E04C0F5D1F840F52
:103BB000951FDC018C9182872F5F253078F38CE094
:103BC000F701CAC08FE89DE00E94B529D80116967A
:103BD0008C911697F701838317969C9117971496EB
:103BE0008C9114978C5F8C7F292F2370822B848378
:103BF0008091AC05868314968C91149783709C7F7A
:103C0000892B878318968C911897808787E0828309
:103C10008DEC81878091CF03882309F481C0A701AF
:103C2000465F5F4F8CE061E00E940E27882309F019
:103C30004DC0D70112968C9112978E5F12968C937D
:103C4000129740C08BEB9DE0288B0E94B529D801CC
:103C500019968C9119978093FF051A968C911A9753
:103C60008093000616968C911697F701838317961A
:103C70009C91179714968C9114978C5F8C7F392F99
:103C80003370832B84838091AC05868314968C914A
:103C9000149783709C7F892B878318968C91189733
:103CA0008087288922838DEC81878091CF038823A8
:103CB000B9F18CE061E04FEF55E00E946124882368
:103CC00029F4D70119961C9219972AC08FEFF70192
:103CD00026C087EE9DE00E94B529D80116968C91EA
:103CE0001697F701838317969C91179714968C91DA
:103CF00014978C5F8C7F292F2370822B8483809173
:103D0000AC05868314968C91149783709C7F892BC5
:103D1000878318968C91808787E0828381EC8187E6
:103D2000D70111961C92119781E060960FB6F89416
:103D3000DEBF0FBECDBFDF91CF911F910F91FF90DE
:103D4000EF90DF90CF90BF90AF909F9008958CEC54
:103D5000F7018187128688E08283E2CF81EB95E0CC
:103D60000895FC018781869586950895982F842F64
:103D7000913099F0913018F0923051F51CC0609359
:103D8000F8053AE0632F0E94052D8093FE05822FEF
:103D90000E94052D8093FA0508956093FD053AE091
:103DA000632F0E94052D80930306822F0E94052D0C
:103DB0008093FC0508956093F7053AE0632F0E9415
:103DC000052D80930206822F0E94052D80931406F4
:103DD00008958091A00308958091D6039091D70310
:103DE000089581E08093D503089581E08093D40302
:103DF000089581E08093D303089581E08093D103F7
:103E000008951F93CF93DF93CDB7DEB7C354D0404F
:103E10000FB6F894DEBF0FBECDBF182F82E590E13C
:103E20000E94B529812F0E942E2A81E693E00E94EC
:103E3000A3298091F5058C8380E18D838091AC0569
:103E40008F838091F40588878C5F8093F40582E0EE
:103E5000898784E08A8782EF8B8787E08C878FE66B
:103E60008D871E878BE08B83CE0101960E94A01365
:103E70001A82CE0101960E94751010939E03CD5BAD
:103E8000DF4F0FB6F894DEBF0FBECDBFDF91CF91ED
:103E90001F9108958091F905982F917080FD08C0B9
:103EA0008091E103882321F01092E10381E00895DD
:103EB0009093E10380E008958091F905982F917027
:103EC00080FF08C08091E203813021F081E080937F
:103ED000E20308959093E20380E008959091F9053C
:103EE000892308950F931F93CF93DF930F92CDB73C
:103EF000DEB78B0189830E945D27898181600E94E2
:103F00007A27882321F40E94712781E00AC080E08B
:103F10000E94A92789830E9471278981F8018083E3
:103F200080E00F90DF91CF911F910F9108951F9323
:103F3000CF93DF9300D0CDB7DEB76A8389830E9429
:103F40005D2789810E947A276A81882321F40E9453
:103F5000712781E009C0862F0E947A27182F0E94BE
:103F6000712781E0111180E00F900F90DF91CF91C8
:103F70001F9108951F93CF93DF930F92CDB7DEB7B4
:103F80008091F805813029F08130E0F08230F1F441
:103F900005C01092DA031092DB0309C08091DA03A6
:103FA0009091FE05891728F48F5F8093DA0311E062
:103FB0000EC08091DB038F5F8093DB039091FA0545
:103FC000891721F41092DA031092DB0310E080913C
:103FD000FD05813029F08130F0F0823001F506C016
:103FE0001092DC031092DD03126019C01260809100
:103FF000DC0390910306891720F48F5F8093DC0324
:104000000EC01D7F8091DD038F5F8093DD03909153
:10401000FC05891721F41092DC031092DD038091D6
:10402000F705813029F08130F0F0823001F506C0CB
:104030001092DE031092DF03146019C014608091A7
:10404000DE0390910206891720F48F5F8093DE03D0
:104050000EC01B7F8091DF038F5F8093DF03909101
:104060001406891721F41092DE031092DF03809169
:10407000A003882311F18CE7BE016F5F7F4F0E9480
:10408000721F8823D1F481E08093D80389818093C3
:10409000F9058F61898310FF02C08D7F898311FF2D
:1040A00003C089818B7F898312FF03C08981877F49
:1040B00089838CE769810E94971F0F90DF91CF91D0
:1040C0001F9108951F93CF93DF9300D0CDB7DEB734
:1040D000162F8CE7BE016F5F7F4F4A830E94721FCD
:1040E0004A81882381F4642F61236161409589812D
:1040F0004823642B69838CE70E94971F91E08823F3
:1041000019F490E001C091E0892F0F900F90DF919A
:10411000CF911F9108951F93CF93DF930F92CDB747
:10412000DEB789830E945D2789810E947A278823D0
:1041300029F089E00E947A27882321F40E947127C0
:1041400081E009C080E00E947A27182F0E94712721
:1041500081E0111180E00F90DF91CF911F910895C0
:10416000CF92DF92EF92FF920F931F93CF93DF9343
:104170000F92CDB7DEB7F82E8B016A010E945D2742
:104180008F2D0E947A27882379F080E00E947A2779
:10419000882351F00E946627EE24E394EF288E2DA9
:1041A0000E947A27882321F40E94712781E02AC087
:1041B00080E00E94A92789830E9471278981F801E4
:1041C00080830E945D278F2D0E947A27882361F0CB
:1041D00081E00E947A27882339F00E9466278E2D7D
:1041E0000E947A27882321F40E94712782E00AC066
:1041F00080E00E94A92789830E9471278981F601A6
:10420000808380E00F90DF91CF911F910F91FF90FD
:10421000EF90DF90CF900895AF92BF92CF92DF9250
:10422000EF92FF920F931F93CF93DF930F92CDB72F
:10423000DEB7182F062F6A01E22EA32E79830E9483
:104240005D27812F880F0E947A277981882391F139
:10425000872F0E947A27882369F1802F0E947A276E
:10426000882341F10E946627812F880F81600E9478
:104270007A278823F9F00E2D1A2DEE24FF245601FB
:104280000894A108B1080FC0EA14FB0411F480E0FF
:1042900001C081E00E94A927F80180830894E11CF5
:1042A000F11C0F5F1F4FEC14FD0471F70E94712782
:1042B00080E003C00E94712781E00F90DF91CF91D1
:1042C0001F910F91FF90EF90DF90CF90BF90AF9034
:1042D0000895EF92FF920F931F93CF93DF93CDB783
:1042E000DEB728970FB6F894DEBF0FBECDBF7C01B6
:1042F00080E560E070E048E050E09E012F5F3F4FB6
:104300000E940C21882309F044C0FE01319697E0F9
:104310002191820F9150E1F781959885891731F0AD
:1043200083E693E00E94A32982E034C00E8110E06E
:1043300083E0000F111F8A95E1F70115110539F18E
:1043400080E5B80145E050E09E012F5F3F4F0E949D
:104350000C218823F1F42A819981920F8B81980F87
:104360003C81930F91953D81931731F089E793E05C
:104370000E94A32984E00EC090E00596080F191F43
:1043800027FFDECFF7011183008380E003C083E0C5
:1043900001C081E028960FB6F894DEBF0FBECDBFF6
:1043A000DF91CF911F910F91FF90EF9008959F9211
:1043B000AF92BF92CF92DF92EF92FF920F931F9333
:1043C000CF93DF93CDB7DEB7C850D1400FB6F89486
:1043D000DEBF0FBECDBF6C01962E5A01FC011082CC
:1043E00080E560E070E048E050E09E012F5F3F4FC5
:1043F0000E940C21882309F06DC0FE01319697E0E0
:104400002191820F9150E1F781959885891709F0E4
:104410005BC00E8110E093E0000F111F9A95E1F749
:104420000115110509F452C080E5B80145E050E0DE
:104430009E012F5F3F4F0E940C21882309F04AC044
:104440008A819981890FEB808E0D9C81890F8195DE
:104450009D818917E9F5FF240B5F1F4F80E5B801A7
:10446000A7019E01275F3F4F0E940C21882391F5F1
:1044700090E00AC049E050E04C0F5D1F240F351F4B
:10448000F9012081920F8F5F282F30E02E153F0514
:1044900088F391958C819817F9F4F60180818F5FEC
:1044A0008083891559F4A114B10441F0F501DE01AE
:1044B00019968DE00D9001928150E1F78A8187FD78
:1044C0000DC00E0D1F1DB0CF82E009C083E007C0F4
:1044D00084E005C081E003C085E001C080E0C85FE2
:1044E000DE4F0FB6F894DEBF0FBECDBFDF91CF9188
:1044F0001F910F91FF90EF90DF90CF90BF90AF9002
:104500009F9008957F928F929F92AF92BF92CF9289
:10451000DF92EF92FF920F931F93CF93DF93CDB76C
:10452000DEB7A1970FB6F894DEBF0FBECDBF85E70B
:104530008B8384E48C8387E58D8383E48E83109260
:10454000CF0332E0E32EF12CEC0EFD1EC70160E03C
:1045500040E050E00E94890A5E010894A11CB11C51
:10456000C50160E040E050E00E94D7218A818823A5
:1045700019F48BE090E106C08981882309F07DC0A1
:1045800084E290E10E94B52911E08CC0872D982D1E
:104590006D2DAE014C5E5F4F0E94890A8DE390E164
:1045A0000E94B5298E010C5E1F4F20E0F801819119
:1045B0008F0129A30E942E2A86E993E00E94A32955
:1045C00029A12F5F2D3091F781E693E00E94A32966
:1045D00011E001E0AA24A3944AC0892D9C2D602FEC
:1045E000AE01495F5F4F0E94D7218A85803351F524
:1045F000112341F188E490E10E94B52927E0E22EE1
:10460000F12CEC0EFD1E10E0F70181917F010E945C
:104610002E2A86E993E00E94A3291F5F1D30A1F78F
:1046200081E693E00E94A329CE014796BE01665F12
:104630007F4F4AE050E00E94412D009711F011E0B9
:1046400001C010E08A85823389F48091CF038823EA
:1046500069F4CE010396BE01645F7F4F44E050E0F1
:104660000E94412D009711F4A092CF030F5F898122
:10467000801708F0B2CFD39407C011E0DD24D394A3
:104680007E2C8F2C9A2CCB2C8A818D1518F011231F
:1046900009F07CCF91E0111190E08091CF03892344
:1046A0008093CF03812FA1960FB6F894DEBF0FBE83
:1046B000CDBFDF91CF911F910F91FF90EF90DF90D1
:1046C000CF90BF90AF909F908F907F9008950F9361
:1046D0001F93CF93DF9300D0CDB7DEB7062F142FF3
:1046E0007A8389830E945D278981880F0E947A27B7
:1046F0007A81882351F0872F0E947A27882329F016
:10470000802F0E947A27882321F40E94712781E05C
:104710000CC0812F0E947A270E9471278FE097E2B8
:104720000197F1F700C0000080E00F900F90DF913B
:10473000CF911F910F910895AF92BF92CF92DF92C8
:10474000EF92FF921F93CF93DF93182F6B015A01C3
:104750007901C0E0D0E00AC0F70141917F01BE01BC
:104760006C0D7D1D812F0E9467232196CA15DB05E4
:1047700099F780E0DF91CF911F91FF90EF90DF904C
:10478000CF90BF90AF900895AF92BF92CF92DF923B
:10479000EF92FF920F931F93CF93DF930F92CDB7BA
:1047A000DEB7082F6A01E22EA32E69830E945D27DF
:1047B000802F880F0E947A2769818823B9F0862F7D
:1047C0000E947A27882391F00E946627802F880F05
:1047D00081600E947A27882349F00E2D1A2DEE243D
:1047E000FF2456010894A108B10813C00E94712744
:1047F00081E015C0EA14FB0411F480E001C081E0FF
:104800000E94A927F80180830894E11CF11C0F5F26
:104810001F4FEC14FD0471F70E94712780E00F9088
:10482000DF91CF911F910F91FF90EF90DF90CF908C
:10483000BF90AF900895CF92DF92EF92FF920F93C7
:104840001F93CF93DF9300D0CDB7DEB77A01690114
:104850006A8389830E945D278981880F0E947A2755
:104860006A81882381F0862F0E947A27882359F055
:104870008601CC24DD240EC0F80181918F010E94B5
:104880007A27882321F40E94712781E00FC00894C1
:10489000C11CD11CCE14DF0479F70E9471278FE070
:1048A00097E20197F1F700C0000080E00F900F90B1
:1048B000DF91CF911F910F91FF90EF90DF90CF90FC
:1048C00008950F931F93CF93DF9300D0CDB7DEB73A
:1048D0008A016A8389830E945D278981880F0E94EB
:1048E0007A276A818823E1F0862F83700E947A27D5
:1048F0008823B1F0F80180810E947A27882381F013
:10490000F80181810E947A27882351F00E94712743
:104910008FE097E20197F1F700C0000080E003C04C
:104920000E94712781E00F900F90DF91CF911F912E
:104930000F9108958091A00380939F032091D90344
:104940002093A0038091D803882389F03091F90542
:104950008091D6039091D70330FF03C08D7F816093
:1049600002C082608E7F9093D7038093D60323305A
:1049700009F442C1243048F480919F03213009F4A6
:104980007BC0223008F0FEC00AC0253009F4C2C145
:10499000253008F43BC1263009F035C207C2882310
:1049A00089F180E490E09093D7038093D6034698F2
:1049B00081E09EE00E94B5298EE09EE00E94B5292C
:1049C0008091D7030E942E2A8091D6030E942E2A1E
:1049D00081E693E00E94A3290E94E2271092E0035F
:1049E00080E060E040E020E00E94B61E81E060E0F0
:1049F00040E020E00E94B61E82E060E040E020E05F
:104A00000E94B61E1092D803359933C00E94EF2839
:104A1000882329F08091E0038F5F8093E0038091E9
:104A2000E003843608F4EFC10E944927882321F46B
:104A300089E19EE00E94B5291092E0038091D6039F
:104A40009091D7038F7B80629093D7038093D60396
:104A500080E061E040E020E00E94B61E0E94DE2778
:104A600085E00E94011F81E08093D9038093D003E9
:104A7000CAC11092E003C7C1813009F449C08CE378
:104A80009EE00E94B52980919F03882389F589E4DF
:104A90009EE00E94B5290E948222882399F480E634
:104AA0009EE00E94B52987E00E94011F8091D603F5
:104AB0009091D70380689093D7038093D60381E0C9
:104AC00060E012C08CE69EE00E94B52988E00E945A
:104AD000011F8091D6039091D70391609093D703E3
:104AE0008093D60381E061E040E020E00E94B61EA2
:104AF00081E89EE00E94B5298091D7030E942E2A6A
:104B00008091D6030E942E2A8CE89EE00E94B5294F
:104B10008091D60387FF31C08091D803882361F04C
:104B20000E944A1F882341F08EE89EE00E94B5292A
:104B300080E00E94011F15C08091D8038823A1F056
:104B40008091D003882381F08091F90580FD0CC00D
:104B500088EA9EE00E94B52980E00E94011F109221
:104B6000D00382E08093D9038091D503882329F074
:104B700084E08093D9031092D503359B44C186EC21
:104B80009EE036C18230A1F08BED9EE00E94B529F7
:104B900088EE9EE00E94B5298091D7030E942E2ABC
:104BA0008091D6030E942E2A81E693E00E94A329D9
:104BB0000E945C1F882351F083EF9EE00E94B5297C
:104BC00081E00E94011F81E08093D903359B09C0D9
:104BD00087E09FE00E94B52986E00E94011F1092A5
:104BE000D9038091D503882309F40DC184E0809313
:104BF000D9031092D50307C180919F03833009F434
:104C000002C18CE19FE00E94B529FDC080919F0305
:104C1000843071F18091D6039091D7038B7F90936C
:104C2000D7038093D60389E29FE00E94B52986E3EB
:104C30009FE00E94B5298091D7030E942E2A80917F
:104C4000D6030E942E2A81E693E00E94A329469A69
:104C50001092E0038091CF03882351F08CE061E053
:104C60004CE953E00E94612481E49FE00E94B52951
:104C70000E94EF28882339F08091E0038F3118F4E7
:104C80008F5F8093E0038091E0038E3159F48CE7CD
:104C900060E040E40E94622082E061E040E020E0C9
:104CA0000E94B61E0E945C1F8823A1F08091D6034B
:104CB0009091D70382608E7F9093D7038093D60321
:104CC0008CE59FE00E94B52981E00E94011F85E0EC
:104CD0008093D9038091D303882319F085E08093D2
:104CE000D903359B90C080E79FE00E94B52986E0FC
:104CF0000E94011F8091CF03882309F47EC08CE0BD
:104D000061E048E953E00E94612485E89FE00E9449
:104D1000B52973C080919F03853041F18BE99FE0F5
:104D20000E94B52988EA9FE00E94B5298091D703A7
:104D30000E942E2A8091D6030E942E2A81E693E0BB
:104D40000E94A32982E060E040E020E00E94B61EBD
:104D50008091CF03882351F08CE061E048E953E073
:104D60000E94612483EB9FE00E94B5298091D303C8
:104D7000882371F08091D6039091D703846090933B
:104D8000D7038093D60382E00E94011F1092D303C1
:104D90008091D403882329F086E08093D903109270
:104DA000D403359B30C089EC9FE022C080919F03E3
:104DB0008630D1F08CE760E440E40E94622046989F
:104DC0008EED9FE00E94B5298BEE9FE00E94B529F1
:104DD0008091D7030E942E2A8091D6030E942E2A0A
:104DE00081E693E00E94A329359B0AC086EF9FE0ED
:104DF0000E94B52986E00E94011F1092D90303C0CA
:104E000081E08093D9038091D103882331F0809190
:104E10009E030E94011F1092D1030895EF92FF920A
:104E20001F93CF93DF930F92CDB7DEB7182F7A0180
:104E300069830E945D27812F880F0E947A276981EC
:104E40008823E9F0862F83700E947A278823B9F09F
:104E50000E946627812F880F81600E947A2788230D
:104E600071F081E00E94A927F701808380E00E9411
:104E7000A927F70181830E94712780E003C00E9467
:104E8000712781E00F90DF91CF911F91FF90EF90FC
:104E900008958BB18F7C8BB98AB18F7C8AB989E0F8
:104EA00094E19A95F1F7549A94E19A95F1F7549810
:104EB0008150B1F789B180720895559A84E18A953D
:104EC000F1F7549A84E18A95F1F70895559884E1B1
:104ED0008A95F1F7549884E18A95F1F70E945D274D
:104EE0000895549884E18A95F1F7559884E18A955C
:104EF000F1F70895F89428E030E090E8492F48232E
:104F000011F4559A01C0559844E14A95F1F7549827
:104F100048E24A95F1F7549A44E14A95F1F796959B
:104F20002150304059F7559884E18A95F1F754980B
:104F300044E14A95F1F799B184E18A95F1F7549AE1
:104F4000559A44E14A95F1F7789481E095FD80E027
:104F50000895282FF894559898E080E0880F34E160
:104F60003A95F1F7549834E13A95F1F74D9981600B
:104F700034E13A95F1F7549A34E13A95F1F79150CA
:104F800069F7222311F0559A01C0559894E19A953A
:104F9000F1F7549838E23A95F1F7549A559A94E11A
:104FA0009A95F1F7789408958091E303882319F096
:104FB0008AE090E0089589E090E0089581E0809390
:104FC000E30308951092E30308958BB18F738BB9B7
:104FD0008AB18F738AB90895579A86E08A95F1F756
:104FE00000C0569A86E08A95F1F700C00895579858
:104FF00086E08A95F1F700C0569886E08A95F1F729
:1050000000C00E94EC270895569886E08A95F1F733
:1050100000C0579886E08A95F1F700C0089528E00F
:1050200030E090E8492F482311F4579A01C057986F
:1050300046E04A95F1F700C056984DE04A95F1F7E1
:105040000000569A46E04A95F1F700C09695215027
:10505000304041F7579886E08A95F1F700C056989E
:1050600096E09A95F1F700C089B146E04A95F1F7CC
:1050700000C0569A579A96E09A95F1F700C080952D
:10508000881F8827881F0895282F579898E080E068
:10509000880F36E03A95F1F700C0569836E03A9519
:1050A000F1F700C04F99816036E03A95F1F700C002
:1050B000569A36E03A95F1F700C0915049F722230D
:1050C00011F0579A01C0579896E09A95F1F700C0F1
:1050D00056983DE03A95F1F70000569A579A96E0B7
:1050E0009A95F1F700C008959091170683B18095C5
:1050F00089279091E403982390959093E40320915D
:10510000E503282329272093E50398239223809100
:105110001706892780931706209116068091170697
:105120008923822B809316062091150680911706FD
:1051300080958923822B809315060895F894909189
:105140001606892390911606982790931606789450
:105150000895F89490911506892390911506982743
:105160009093150678940895F89490911706789482
:10517000892308958093EA0381E08093E9030895E9
:105180001092E903089581E09091E903992309F4CD
:1051900080E008958091EA03882329F0815080936C
:1051A000EA0380E0089581E008958093E80381E0B8
:1051B0008093E70308951092E703089581E09091AA
:1051C000E703992309F480E0089581E09091E803D2
:1051D000911180E0089581E08093E6030895809125
:1051E000E603882321F01092E60381E0089580E031
:1051F00008951092C5008CE08093C40088E98093E4
:10520000C10010929A061092980610929906109278
:105210001B0708959091980620919A0691509F77C8
:105220002917C1F3E0919A06F0E0E556F94F808323
:1052300080919A068F5F80939A0680919A068038B3
:1052400011F410929A068091C10080628093C1008F
:1052500008953091990620911B073217A1F02091F3
:105260001B07E22FF0E0E85EF94F3081FC0130834C
:105270002F5F20931B0780911B07803831F4109219
:105280001B0780E0089581E0089580E008951F9253
:105290000F920FB60F920BB60F9211248F939F931C
:1052A000EF93FF93E0919806F0E0E556F94F808187
:1052B0008093C600809198068F5F809398068091B6
:1052C0009806803811F41092980690919A06809171
:1052D0009806981729F48091C1008F7D8093C100B2
:1052E000FF91EF919F918F910F900BBE0F900FBE8A
:1052F0000F901F9018951F920F920FB60F920BB63A
:105300000F9211248F939F93EF93FF9380919906AF
:10531000E82FF0E09091C600E85EF94F90838F5F30
:105320008093990680919906803811F4109299061D
:10533000FF91EF919F918F910F900BBE0F900FBE39
:105340000F901F901895CF93DF93EC0108C08A301F
:1053500019F48DE00E940A2989910E940A29888106
:105360008823A9F7DF91CF9108951F93CF93DF93FF
:10537000EC012196FC0114911A3019F48DE00E9481
:105380000A29812F0E940A29FE01219614911123D6
:1053900099F7DF91CF911F9108950F931F93CF93AA
:1053A000DF93082FC8E0D0E010E8812F802311F0B0
:1053B00081E301C080E30E940A2916952197A9F78D
:1053C000DF91CF911F910F910895DF92EF92FF929D
:1053D0000F931F93CF93DF93CDB7DEB729970FB607
:1053E000F894DEBF0FBECDBF8C01DE011196E1EA5D
:1053F000F3E088E001900D928150E1F77E0108947E
:10540000E11CF11C84E0D82E91E010C08F5F021BDC
:10541000130B90E002171307C8F7992329F4805D56
:1054200099870E940A299985DA9431F0F701219130
:1054300031917F0180E0EECF802F805D0E940A29AC
:1054400029960FB6F894DEBF0FBECDBFDF91CF9186
:105450001F910F91FF90EF90DF9008951F93CF93CE
:10546000DF93CDB7DEB760970FB6F894DEBF0FBEFF
:10547000CDBF182FDE011196E9EAF3E080E101903B
:105480000D928150E1F7812F82958F70E1E0F0E07D
:10549000EC0FFD1FE80FF11D80810E940A291F708B
:1054A000E1E0F0E0EC0FFD1FE10FF11D80810E94B3
:1054B0000A2960960FB6F894DEBF0FBECDBFDF910C
:1054C000CF911F910895CF93DF93CDB7DEB7C3542B
:1054D000D0400FB6F894DEBF0FBECDBFA89528E22E
:1054E00088E190E00FB6F894A895809360000FBE15
:1054F000209360001092A7051092A8051092A905AC
:105500001092AA051092AD050E94F9280E94540835
:105510000E94E5270E94AE1E9093B0058093AF05D0
:1055200089E0809381008FE39FE1909389008093CD
:10553000880082E080936F002C9885B1806685B9E1
:1055400084B1806784B94098389A139A149881B1CD
:10555000886181B915980D9A46983E9A5A9A5B9837
:1055600080E060E144E054E02CE034E00E949910D7
:1055700081E060E244EF53E02CE134E00E949910B6
:1055800082E060E44CEF53E024E134E00E949910A3
:105590001092AB0578948FEF9FE00E94672D082F43
:1055A0008F3F31F48FEF9FE060E00E94792D00E0A3
:1055B00083EF93E00E94B5298BE094E00E94B52927
:1055C000802F0E942E2A8AE194E00E94B52982B1A0
:1055D0008C7F82B900FD119A01FD109A1092A605E8
:1055E0008CE194E00E94B52984E394E00E94B529FF
:1055F000809160000E942E2A8DE394E00E94B529DC
:105600008FE394E00E94B5298BE193E00E94A329E7
:1056100088E494E00E94B5298EE594E00E94B529C3
:1056200084E694E00E94B52984E794E00E94B529BD
:105630008AE794E00E94B52985E894E00E94B529A4
:105640008EE894E00E94B52983E994E00E94B52990
:105650008FE994E00E94B52983EA94E00E94B5297D
:105660008CEA94E00E94B5298EEA94E00E94B52964
:1056700084B70E942E2A86EB94E00E94B52914BEBE
:105680000E9458138093AC050E94DD0E81E293E0E6
:105690000E94A3298091AC050E942E2A82E393E008
:1056A0000E94A3290E94CE0D80E28093F5051092FE
:1056B000F60500E010E085E0F82EEE24EA9425E0FF
:1056C000D22EA8950E94070E0E941C098091A20567
:1056D000882371F080E96FE975E00E94C61282E9C3
:1056E00064EA75E00E94C612F110FA941092A205C5
:1056F000FF2011F40E949A248091A305882321F0B1
:105700000E94BA1F1092A3050E94ED0E882311F487
:105710000E945D0F8091AF059091B005FC01208142
:1057200020FF2AC00E94CD13E091AF05F091B00593
:1057300090819E7F90838823F9F4CF010E949A1371
:105740002091AF053091B005882389F4C901BE01CD
:105750006F5F7F4F0E94F413882371F0CE01019692
:105760000E94A013CE0101960E94751005C0C901C8
:105770000E94B11E0E9493108091AE05882309F407
:10578000A0CF0E94C328882379F00E94CA288823CA
:1057900059F081E08093AB050E94C02888EB94E02B
:1057A0000E94B52900E010E08091A7059091A8051E
:1057B000A091A905B091AA050196A11DB11D8093E4
:1057C000A7059093A805A093A905B093AA0580E02A
:1057D0000E94501181E00E94501182E00E945011FD
:1057E0008091AB05843009F460C0853040F481308D
:1057F000E9F0813070F0833009F09EC037C0863008
:1058000009F488C0863008F46DC0873009F094C070
:1058100083C081B18C7F81B98AB1837F8AB90D9AA7
:10582000389A139A14981092AD0586C080E00E94B1
:10583000C808F2E08C3B9F0708F47EC00F5F1F4F43
:105840000230110509F078C083E08093AB0513980E
:10585000149A82ED94E00E94B5298091A705909159
:10586000A8050E94E5298BEF94E01CC005301105C6
:1058700019F481B1836081B90F5F1F4F05311105A4
:1058800008F45AC0389884E08093AB058EEF94E01A
:105890000E94B5298091A7059091A8050E94E5294D
:1058A0008EE295E00E94B52945C0319B45C00F5F4F
:1058B0001F4F0630110508F43FC00D988AB18C6067
:1058C0008AB9D092AB0581E395E00E94B529809119
:1058D000A7059091A8050E94E5298FE595E00E9413
:1058E000B5292AC08091AD05882331F582E695E07F
:1058F0000E94B5298091A7059091A8050E94E529ED
:1059000085E795E00E94B5290E94630E81E08093AF
:10591000AD0512C00D9A10C0389A0D9A8AB1837FD6
:105920008AB9139A149881E08093A6051092AB056A
:105930001092AD0500E010E0C090AB05EC1409F446
:1059400041C022E0C216B9F02C1530F081E0CC2025
:1059500071F0C816B9F50AC0E5E0CE16E1F0F7E03F
:10596000CF1621F124E0C21669F50AC081E060E09B
:1059700041E050E01FC081E060E042E050E01AC02A
:1059800081E060E040E050E00E94B31082E060E01F
:1059900042E050E015C081E060E040E050E00E944D
:1059A000B31082E060E041E050E00AC081E060E0D6
:1059B00040E050E00E94B31082E060E040E050E040
:1059C0000E94B3101092AE05EC2C7BCE629FD001EA
:1059D000739FF001829FE00DF11D649FE00DF11DAA
:1059E000929FF00D839FF00D749FF00D659FF00D59
:1059F0009927729FB00DE11DF91F639FB00DE11D46
:105A0000F91FBD01CF0111240895991B79E004C04D
:105A1000991F961708F0961B881F7A95C9F78095ED
:105A2000089597FB092E07260AD077FD04D00CD0E5
:105A300006D000201AF4709561957F4F0895F6F70F
:105A4000909581959F4F0895AA1BBB1B51E107C0FC
:105A5000AA1FBB1FA617B70710F0A61BB70B881FFE
:105A6000991F5A95A9F780959095BC01CD0108958D
:105A7000FB01DC0102C005900D9241505040D8F767
:105A80000895FB01DC0104C08D910190801921F47F
:105A900041505040C8F7881B990B0895FB01DC0169
:105AA00002C001900D9241505040D8F70895DC019A
:105AB000CB01FC01F999FECF06C0F2BDE1BDF89A19
:105AC000319600B40D9241505040B8F70895F999BD
:105AD000FECF92BD81BDF89A992780B50895DC016B
:105AE000CB0103C02D910E947A2D41505040D0F738
:105AF0000895262FF999FECF1FBA92BD81BD20BD12
:105B00000FB6F894FA9AF99A0FBE01960895F89490
:025B1000FFCFC5
:105B12000A0001FFFF204552524F5221003A203025
:105B220078000A002E2E2E204552524F52210A0092
:105B32002E2E2E20646F6E65210A00646F6E652121
:105B42000A00205265616420556E697175652D49A0
:105B5200443A200020525F4552524F522100206D9C
:105B6200560A0020000A0A383330303E0A00756EA9
:105B72006B6E6F776E20636F6D6D616E640A0038B5
:105B82003330303E00535441540048454C5000528B
:105B9200544D310052544D320052544D3300525440
:105BA2004D340052544D350052544D360052544D2E
:105BB200370052544D3800564F4C540050524F4DFE
:105BC2000049440044414357004441435200007598
:105BD20002820D7A02960B7F025B0D8402340D89DC
:105BE20002220D8E02190D9302100D9802070D9DCF
:105BF20002900BA202C80CA702720CAC02160CB1E6
:105C020002300CB402C70BB9029C0BBE0200000AA0
:105C120000726571206F75742064726F70706564B4
:105C220020616674657220330A000A322E372E31E3
:105C3200004D6F64756C6520416464726573733ADC
:105C420020000A0A000A006F6666733A0020636E3B
:105C5200743A002000322E372E31006D065306C4EE
:105C6200071306840744070407D3059305C4068473
:105C7200060A0072746D20636D6E20686472206380
:105C8200686B206661696C0A006D756C74206865CA
:105C92006164657220636865636B73756D206572FC
:105CA200726F72210A00200020002FFC2C1C06FFBC
:105CB200FF1027E80364000A0030313233343536EE
:0A5CC200373839414243444546009B
:00000001FF
